:100000000C9438050C9481050C9486060C9481059B
:100010000C9481050C9481050C9481050C94810548
:100020000C9481050C9481050C94700D0C94460E73
:100030000C94351D0C9481050C9481050C9481055C
:100040000C9481050C9481050C9481050C94810518
:100050000C9481050C94A91D0C9481050C948105C8
:100060000C9481050C9481050C9481050C948105F8
:100070000C9481050C9481050C9481050C948105E8
:100080000C9481050C9481050C9481050C948105D8
:100090000C9481050C948105A507B807D107D507F5
:1000A000D907DC07E207E607EA07EE07F207B70E13
:1000B000D90EC70FD90EC70F1E0F410FC70F960FCE
:1000C000A90FFE12FE122D132D138B13C913E31566
:1000D000E315E213E315E314E314B715E315E31591
:1000E000CE1500291E1F20212223242526272D2E50
:1000F0002A2B141A0815171C180C12132F3028E07D
:10010000041607090A0B0D0E0F333435E1311D1BA0
:100110000619051110363738E555E22C393A3B3CC3
:100120003D3E3F4041424353475F6061565C5D5EE8
:1001300057595A5B626358E4544445E6ABE3E765BC
:10014000A5A6A8B4B0A7AFB6BCBBBAB9B8B5B3B290
:10015000AC4A524BAA50A94FB74D514E494C464854
:100160000000706275663A2066756C6C0A00253076
:10017000325820004B6579626F617264207374613C
:1001800072742E0A0055534220636F6E666967755C
:100190007265642E0A000D0A696E69740A005B4478
:1001A0005D005B435D002C035800540020006B0091
:1001B0006500790062006F00610072006400200039
:1001C00063006F006E0076006500720074006500C9
:1001D000720000000E0374002E006D002E006B00F4
:1001E0002E0000000403090409028D00050100A08F
:1001F000320904000001030101000921110100017D
:100200002240000705810308000A090401000103D8
:10021000010200092111010001224D00070582039E
:1002200008000A090402000103000000092111016D
:1002300000012236000705830308000A09040300B1
:10024000020300000009211101000122220007051C
:1002500084032000010705040320000109040400B1
:1002600001030000000921110100012239000705E6
:1002700085032000011201100100000008EDFE12AC
:100280006501000102000105010906A10105071928
:10029000E029E71500250195087501810205081977
:1002A00001290595057501910295017503910105D7
:1002B00007190029F71500250195F875018102C07D
:1002C0000631FF0974A1010975150026FF0095206C
:1002D000750881020976150026FF009520750891A2
:1002E00002C005010980A101850216810026B70020
:1002F0001A81002AB700751095018100C0050C090C
:1003000001A1018503160100269C021A01002A9C06
:1003100002751095018100C005010902A1010901C2
:10032000A10005091901290515002501950575018B
:10033000810295017503810105010930093115819B
:10034000257F95027508810609381581257F95015D
:1003500075088106050C0A38021581257F950175FF
:10036000088106C0C005010906A101050719E02999
:10037000E715002501950875018102950175088131
:100380000105081901290595057501910295017569
:100390000391010507190029FF150026FF009506A6
:1003A00075088100C0636F6E73756D65723A2025A4
:1003B0003034580A0073797374656D3A20253034EF
:1003C000580A000A002530325820006B6579626FA8
:1003D0006172643A20004C45443A20253032580A74
:1003E00000253032583A202530386225730A0072D1
:1003F0002F632030313233343536370A0064656C70
:100400005F6B65795F6269743A2063616E2774205F
:1004100064656C3A20253032580A006164645F6B71
:1004200065795F6269743A2063616E277420616444
:10043000643A20253032580A00290A002575002F19
:10044000002575005D28002564002000256400203B
:100450000025640020002564007C0025303258000F
:100460006D6F7573656B6579205B62746E7C782047
:1004700079207620685D287265702F61636C293A57
:10048000205B006D6B5F776865656C5F74696D6597
:100490005F746F5F6D6178203D2025640A006D6B8D
:1004A0005F776865656C5F6D61785F7370656564C3
:1004B000203D2025640A006D6B5F74696D655F7473
:1004C0006F5F6D6178203D2025640A006D6B5F6D64
:1004D00061785F7370656564203D2025640A006D56
:1004E0006B5F696E74657276616C203D2025640ACD
:1004F000006D6B5F64656C6179203D2025640A00A6
:100500006D6B5F776865656C5F74696D655F746F4F
:100510005F6D6178203D2025640A006D6B5F776810
:1005200065656C5F6D61785F7370656564203D2003
:1005300025640A006D6B5F74696D655F746F5F6D34
:100540006178203D2025640A006D6B5F6D61785FE6
:100550007370656564203D2025640A006D6B5F69DA
:100560006E74657276616C203D2025640A006D6BA7
:100570005F64656C6179203D2025640A000A0025CE
:100580007500363A20776865656C5F74696D655FE4
:10059000746F5F6D61783A20000A00257500353A66
:1005A00020776865656C5F6D61785F737065656401
:1005B0003A20000A00257500343A2074696D655FA1
:1005C000746F5F6D61783A20000A00257500333A38
:1005D000206D61785F73706565643A20000A0025BC
:1005E0007500323A20696E74657276616C286D739D
:1005F000293A20000A00257500313A2064656C61B3
:1006000079282A31306D73293A20000A092D2056A5
:10061000616C756573202D0A004D3E004D25643ECA
:1006200020003F007365742064656661756C740A10
:1006300000433E200077686572652064656C7461D4
:100640003A20637572736F723D25642C207768655C
:10065000656C3D25640A53656520687474703A2F93
:100660002F656E2E77696B6970656469612E6F7294
:10067000672F77696B692F4D6F7573655F6B657950
:10068000730A000A092D204D6F7573656B6579201B
:100690002D0A4553432F713A09717569740A313A2D
:1006A0000964656C6179282A31306D73290A323A00
:1006B00009696E74657276616C286D73290A333A24
:1006C000096D61785F73706565640A343A0974690D
:1006D0006D655F746F5F6D61780A353A097768659B
:1006E000656C5F6D61785F73706565640A363A09A1
:1006F000776865656C5F74696D655F746F5F6D6168
:10070000780A0A703A097072696E742076616C75A5
:1007100065730A643A097365742064656661756C73
:1007200074730A75703A092B310A646F776E3A094F
:100730002D310A706775703A092B31300A70676481
:100740006F776E3A092D31300A0A7370656564203F
:100750003D2064656C7461202A206D61785F737040
:10076000656564202A2028726570656174202F20D9
:1007700074696D655F746F5F6D6178290A003F0071
:100780004D3E2000433E20004C25640A000A092DFE
:1007900020436F6E736F6C65202D0A4553432F7194
:1007A0003A09717569740A6D3A096D6F7573656BF5
:1007B00065790A000A092D204D61676963202D0AB9
:1007C000643A0964656275670A783A096465627516
:1007D00067206D61747269780A6B3A0964656275A5
:1007E00067206B6579626F6172640A6D3A096465AE
:1007F000627567206D6F7573650A763A0976657262
:1008000073696F6E0A733A097374617475730A635E
:100810003A09636F6E736F6C65206D6F64650A30A3
:100820002D343A096C61796572302D3428463130A7
:100830002D4634290A506175733A09626F6F746CE2
:100840006F616465720A6E3A094E4B524F0A003F5F
:10085000004E4B524F3A206F66660A004E4B524F85
:100860003A206F6E0A0074696D65725F726561642B
:10087000333228293A202530346C580A006B6579C8
:10088000626F6172645F6E6B726F3A2025580A0066
:100890006B6579626F6172645F69646C653A20258B
:1008A000580A006B6579626F6172645F70726F7471
:1008B0006F636F6C3A2025580A00686F73745F6B22
:1008C0006579626F6172645F6C65647328293A2090
:1008D00025580A000A092D20537461747573202D60
:1008E0000A004743433A20342E392E3220415652D3
:1008F0002D4C4942433A20312E382E3073766E20EB
:100900004156525F415243483A2061767235310A6E
:10091000004F5054494F4E533A204C554641204DBC
:100920004F5553454B45592045585452414B455915
:1009300020434F4E534F4C4520434F4D4D414E4465
:10094000204E4B524F20313032340A004255494C30
:10095000443A20653131333433342D64697274790B
:10096000202832313A35323A3236204D6172203108
:10097000342032303138290A005649443A20307840
:100980004645454428742E6D2E6B2E29205049442F
:100990003A20307836353132285854206B657962E8
:1009A0006F61726420636F6E766572746572292060
:1009B0005645523A203078303030310A00444553A1
:1009C000433A20636F6E76657274205854206B65CD
:1009D00079626F61726420746F205553420A000A75
:1009E000092D2056657273696F6E202D0A000A6DFD
:1009F0006F7573653A206F66660A000A6D6F7573CE
:100A0000653A206F6E0A000A6B6579626F617264E5
:100A10003A206F66660A000A6B6579626F617264DC
:100A20003A206F6E0A000A6D61747269783A206F1D
:100A300066660A000A6D61747269783A206F6E0A00
:100A4000000A64656275673A206F6E0A000A646581
:100A50006275673A206F66660A000A0A626F6F74F1
:100A60006C6F616465722E2E2E2000433E200000C4
:100A700011241FBECFEFD0E2DEBFCDBF04B603FE10
:100A800027C08091CF029091D002A091D102B09165
:100A9000D2028730904BA740B04BD1F41092CF02D6
:100AA0001092D0021092D1021092D20214BE84B7DA
:100AB000877F84BF0FB6F894A89580916000886105
:100AC00080936000109260000FBEE0E0FEEF099599
:100AD00011E0A0E0B1E0E2EAFDE400E00BBF02C0FB
:100AE00007900D92A833B107D9F722E0A8E3B1E04F
:100AF00001C01D92AF3CB207E1F70E94940A0C942A
:100B0000CF260C940000FF93EF93E0913801F09111
:100B10003901309709F00995EF91FF910895FC0193
:100B20008591803011F0EFDFFBCF0895FF27E0E2E1
:100B300030E247FF0CC0419597FF09C0EDE2609598
:100B4000709580959095611D711D811D911D27FFE8
:100B500002C0219530E350E2AA27660F771F881F55
:100B6000991FAA1FA41710F0A41B63955A95A9F703
:100B7000AA3008F0A95FA05DAF93F39561157105E8
:100B80008105910541F7ED3211F4EF93F395F217DA
:100B900018F43F93F395FBCF8F91B5DFFA95E1F70A
:100BA0000895E991F9918591803021F0853219F00D
:100BB000AADFF9CF089520E0E89455915532C1F3AA
:100BC000503311F4689455915A3348F4505390F3CC
:100BD000220F022E220F220F200D250FF4CF0EF42C
:100BE000219589919991533619F3533729F153354A
:100BF00059F1BC0188279927E8945C3621F4899142
:100C0000999168945591543639F446EF7EF077FF08
:100C10000DC08FEF9FEF0AC055374AE039F05835C5
:100C200040E121F0523642E009F00895FF93EF933E
:100C30007DDFEF91FF91B7CFFF93EF93FC0181919F
:100C40008030B9F360DFFBCFFF93EF9368DFF1CF24
:100C5000DF93CF93CDB7DEB72596A3DFCF91DF919A
:100C60000895E9E6F0E0808188608083E9982F9814
:100C7000279A2FEF89E698E1215080409040E1F7D4
:100C800000C0000027985898509A5998519A2FEF11
:100C900089EF90E0215080409040E1F700C00000D3
:100CA0005198599A5098589AE19AE99A08954FB7ED
:100CB000F89420913E0130913F0180913C01909148
:100CC0003D014FBF28173907F9F09FB7F8942091DD
:100CD0003C0130913D0140913E0150913F0142174E
:100CE000530779F0F901EE0FFF1FE05CFE4F8081A2
:100CF0002F5F3F4F2F71332730933D0120933C01ED
:100D000001C080E09FBF089580E008951F920F9278
:100D10000FB60F9211240BB60F922F933F934F9360
:100D20005F936F937F938F939F93AF93BF93CF9373
:100D3000EF93FF9329B1217090913B01992319F012
:100D4000993058F403C0211108C037C080913A018E
:100D500086952111806880933A0181E0890F809304
:100D60003B01983051F540913A0150E0CFB7F894EB
:100D700080913E0190913F019C012F5F3F4F2F7169
:100D8000332760913C0170913D012617370761F0D0
:100D9000880F991FFC01E05CFE4F51834083309324
:100DA0003F0120933E0104C082E691E00E948F053E
:100DB000CFBF10923B0110923A01FF91EF91CF917A
:100DC000BF91AF919F918F917F916F915F914F9163
:100DD0003F912F910F900BBE0F900FBE0F901F9061
:100DE0001895803389F1A0F48E3138F48C3140F5B8
:100DF000803181F1893111F10895843219F128F49B
:100E000090EE980F9330F0F008958E32E9F0089547
:100E10008A3448F48734E0F48533C1F08833B1F084
:100E20008233C9F411C08D3499F018F48B3481F0F9
:100E3000089591EB980F953058F008958AE508953C
:100E4000885C0895805C08958C5B08958F5D08959B
:100E5000885D08958EE60895CF93DF93D82FD770DD
:100E6000C82FC695C695C6956D2F8C2F0E944C1124
:100E7000882371F0EC2FF0E0EF57FE4F81E090E017
:100E800001C0880FDA95EAF78095908189238083E5
:100E9000DF91CF910895CF93DF93D82FD770C82FCC
:100EA000C695C695C6956D2F8C2F0E944C11811149
:100EB0000DC0EC2FF0E0EF57FE4F81E090E001C055
:100EC000880FDA95EAF79081892B8083DF91CF91A3
:100ED00008958091B10281608093B1020E94310631
:100EE000E1E8F1E080E18E0F11928E13FDCF0895BD
:100EF000CF93DF931F92CDB7DEB765E08FE00E94FE
:100F00004C11882319F08DE70E942C070E94570688
:100F1000882371F01F928F932EE631E03F932F9339
:100F200089830E9428060F900F900F900F9089815F
:100F3000E09180014E2F50E04B30510508F058C031
:100F4000FA01E45BFF4F0C94B226803E21F0813E13
:100F500021F486E014C081E012C01816BCF09FE7AF
:100F6000980F9E3708F044C080580E942C0740C05C
:100F70008A3221F0873B31F484E001C082E0809323
:100F8000800138C018162CF40E94F1060E944B070D
:100F90002FC09FE7980F9E3758F580580E94F106A2
:100FA000E4CF803E29F583E0EACF873309F58CE76B
:100FB0001CC0803EE9F41EC08A3AD1F48CE70E943E
:100FC0002C0718C08D31A1F487E0D9CF853481F486
:100FD00088E0D5CF813E61F489E0D1CF8D3941F4ED
:100FE0008AE0CDCF853C21F48DE70E944B0702C0FB
:100FF0001092800181E00F90DF91CF910895E82F4A
:10100000F0E0EF57FE4F80810895E1E8F1E080E1E4
:101010008E0F11928E13FDCF089508958091B50122
:1010200008959FB7F894109294019FBF9091C602C3
:10103000943009F057C09091E9009F703091EC0016
:10104000232F217030FD20E8922B24E02093E9002B
:101050002091EB0020FF43C02091EE0027FF3FC00E
:1010600020919101222321F02091E80025FF37C033
:101070001092910126E03091E80035FD15C03091C5
:10108000C602343061F53091EB0035FD28C02150A7
:1010900021F481E08093910122C0EFE9FFE03197D4
:1010A000F1F700C00000E7CF8093F1008091E800E5
:1010B00085FD0AC08091E80080FFFCCF8091E800A8
:1010C0008E778093E80006C08FB7F89421E02093D4
:1010D00094018FBF9F709093E90080E008959F7006
:1010E0009093E9008FEF0895CF93DF9300D01F9284
:1010F000CDB7DEB79C018091C602843019F593E02C
:1011000099833B832A839093E9008FEF9091E800C5
:10111000815095FD06C095ED9A95F1F7000081117B
:10112000F5CF8091E80085FF0DC040E050E063E01E
:1011300070E0CE0101960E94610B8091E8008E77ED
:101140008093E8000F900F900F90DF91CF9108955A
:10115000CF93DF9300D01F92CDB7DEB72091C602A8
:10116000243021F522E029839B838A8383E08093C6
:10117000E9008FEF9091E800815095FD06C095ED54
:101180009A95F1F700008111F5CF8091E80085FF75
:101190000DC040E050E063E070E0CE0101960E9497
:1011A000610B8091E8008E778093E8000F900F909C
:1011B0000F90DF91CF9108952091C6022430F1F471
:1011C00022E02093E9002FEF3091E800215035FD17
:1011D00006C035ED3A95F1F700002111F5CF2091C9
:1011E000E80025FF0BC040E050E065E070E00E94A1
:1011F000610B8091E8008E778093E8000895CF938B
:10120000DF932091C602243009F048C0EC018091A0
:101210000A018823E1F080910B018823C1F085E069
:101220008093E9008FEF9091E800815095FD06C012
:101230009AE29A95F1F700C08111F5CF8091E8000C
:1012400085FF2CC040E050E060E270E017C081E014
:101250008093E9008FEF9091E800815095FD06C0E2
:1012600095ED9A95F1F700008111F5CF8091E80096
:1012700085FF14C040E050E068E070E0CE010E94BD
:10128000610B8091E8008E778093E80080E2FE0198
:10129000A5E9B1E001900D928A95E1F7DF91CF9138
:1012A000089582EA91E00E948F058091C502811124
:1012B00009C00E94F20C0E94540D8091E2008460EB
:1012C0008093E20008958EE991E00E948F051092CC
:1012D000C50208950895209192012F5F822F62E345
:1012E0000E949226992319F020939201089510925A
:1012F000920180919401882371F18091C60284301B
:1013000041F58091E9008F702091EC00922F91704F
:1013100020FD90E8892B94E09093E9009091EB00F8
:1013200090FF14C09091EE0097FF10C09091E800DC
:1013300095FF03C01092F100F9CF9091E80090FF63
:1013400005C09091E8009E779093E8008F7080939D
:10135000E90010929401089542E061EC81E00E945E
:101360006C0C42E061EC82E00E946C0C42E061ECAB
:1013700083E00E946C0C42E261EC84E00E946C0C01
:1013800042E261EC85E00C946C0C8091C8028330E1
:1013900009F455C030F4813071F0823009F48EC008
:1013A00008958A3009F47AC08B3009F460C089301E
:1013B00009F09CC020C08091C702813A09F096C014
:1013C0008091E800877F8093E8008091CB02909124
:1013D000CC02892B21F460E285E991E003C060E052
:1013E00080E090E070E00E94AC0B8091E8008B7789
:1013F0008093E80008958091C702813209F076C099
:101400008091CB029091CC02009719F0049709F0DB
:101410006DC08091E800877F8093E8008091E800AC
:1014200082FD05C08091C6028111F8CF5FC0809116
:10143000F1008093B5018091E8008B7753C08091D3
:10144000C702813A09F052C08091CB029091CC0240
:10145000892B09F04BC08091E800877F8093E800DA
:101460008091E80080FFFCCF80910A0136C0809116
:10147000C7028132D9F58091CB029091CC02892BA1
:10148000A9F58091E800877F8093E8000E94A10C75
:101490008091C90280930A010C9405168091C702BD
:1014A000813221F58091E800877F8093E8000E94D7
:1014B000A10C8091CA028093B60108958091C70261
:1014C000813AA1F48091E800877F8093E8008091C1
:1014D000E80080FFFCCF8091B6018093F1008091FD
:1014E000E8008E778093E8000C94A10C089508958D
:1014F00008958091B501809393011092B50180E029
:101500000E940D080E9405080C9405160C94790A97
:101510000E94F41C8091C402882329F00E941D1DA2
:1015200081110C944B0B089584B7877F84BF0FB64D
:10153000F894A89580916000886180936000109273
:1015400060000FBE90E080E80FB6F89480936100D1
:10155000909361000FBE81E198E00E94C51C86E96E
:1015600091E00E948F050E94770A0E94A0100E94BD
:10157000F20C0E94540D8091E20084608093E2009E
:1015800078948091C6028430E1F781ED97E001976D
:1015900039F0EFE9FFE03197F1F700C00000F7CF35
:1015A00085E891E00E948F050E94A21080E091E002
:1015B0000E94DF0F84E791E00E948F050E94780A65
:1015C0008091C602853019F40E94880AF9CF0E94E2
:1015D000A610F6CF0E94311D809193018093B50132
:1015E00008950C94EA0A292F332723303105C9F0D6
:1015F00064F42130310581F02230310509F043C017
:101600008DE890E028EE31E042C021323105F1F062
:101610002232310541F137C082E190E025E732E026
:1016200036C099278130910541F08230910541F013
:10163000892B49F5E4EEF1E005C0E4EDF1E002C0EC
:10164000E6EAF1E0849190E09F0121C06530D8F492
:10165000E62FF0E0EE0FFF1FED5DFE4F20813181A0
:1016600089E090E014C0653070F470E0FB01EE0F8B
:10167000FF1FE75EFE4F20813181FB01EC5EFE4FD4
:10168000808190E004C080E090E020E030E0FA014A
:1016900031832083089584E189BD86E189BD09B441
:1016A00000FEFDCF8091D8008F7D8093D80080917F
:1016B000E00082608093E0008091E00081FDFCCF3B
:1016C0000895CF92DF92EF92FF920F931F93CF93E3
:1016D000DF93EC018B016A010E94C00C811133C0C1
:1016E000C114D10439F0F60180819181081B190BD6
:1016F000C80FD91FE12CF12C0115110519F18091AA
:10170000E80085FD16C08091E8008E778093E800A0
:10171000C114D10449F0F60180819181E80EF91ECF
:10172000F182E08285E00FC00E94C00C882321F383
:101730000AC089918093F10001501109FFEFEF1A5F
:10174000FF0ADACF80E0DF91CF911F910F91FF90D8
:10175000EF90DF90CF9008952091CD023091CE028E
:101760002617370748F06115710539F42091E80014
:101770002E772093E80001C0B90140E061157105A2
:1017800099F12091C602222309F441C0253009F4C1
:1017900040C02091E80023FD3EC02091E80022FDDA
:1017A00030C02091E80020FFE9CF2091F200309175
:1017B000F300FC01CF016115710559F028303105A6
:1017C00040F481918093F100615071092F5F3F4F88
:1017D000F1CF41E02830310509F040E02091E800E8
:1017E0002E772093E800CACF4111CBCF0AC0809159
:1017F000C602882361F0853061F08091E80083FDA6
:101800000AC08091E80082FFF2CF80E0089582E074
:10181000089583E0089581E008952091CD023091EC
:10182000CE022617370748F06115710539F420916B
:10183000E8002E772093E80001C0B901FC0120E008
:101840006115710581F18091C602882309F43EC0BB
:10185000853009F43DC08091E80083FD3BC0809154
:10186000E80082FD2DC08091E80080FFE9CF8091E3
:10187000F2009091F3006115710559F088309105DF
:1018800040F424912093F100319661507109019642
:10189000F2CF21E0089709F020E08091E8008E77F0
:1018A0008093E800CDCF2111CECF0AC08091C6022F
:1018B000882361F0853061F08091E80083FD0AC0E3
:1018C0008091E80082FFF2CF80E0089582E00895E1
:1018D00083E0089581E00895982F973058F590930C
:1018E000E900981739F07091EC002091ED005091CB
:1018F000F00003C0242F762F50E021FF19C0309153
:10190000EB003E7F3093EB003091ED003D7F309354
:10191000ED003091EB0031603093EB007093EC0000
:101920002093ED005093F0002091EE0027FF07C0B8
:101930009F5FD3CF8F708093E90081E0089580E0AE
:1019400008958091C70287FF11C08091E80082FD51
:1019500005C08091C6028111F8CF11C08091E800C6
:101960008B770BC08091C602882349F08091E800F4
:1019700080FFF8CF8091E8008E778093E80008958B
:101980002091E4003091E50095E64091EC00842F31
:10199000817040FF22C08091E80080FD1CC08091D2
:1019A000C602882391F0853091F08091EB0085FD8F
:1019B00010C04091E4005091E5004217530729F30D
:1019C0009A01915011F784E0089582E0089583E030
:1019D000089581E0089580E008954091E80042FF75
:1019E000DECF08950E94630D0E946B0DE0EEF0E0E3
:1019F000808181608083E8EDF0E080818F77808353
:101A000019BCA7EDB0E08C918E7F8C9380818F7E86
:101A100080831092C50208950F931F93CF93DF9395
:101A20000E94630D0E946B0DC8EDD0E088818F7716
:101A3000888388818068888388818F7D8883E7EDAB
:101A4000F0E080818068808319BC1092C6021092F9
:101A5000C2021092C4021092C30200EE10E0F8011C
:101A600080818B7F808388818160888342E060E011
:101A700080E00E946C0CE1EEF0E080818E7F80833C
:101A8000E2EEF0E0808181608083808188608083E5
:101A9000F80180818E7F8083888180618883DF91D7
:101AA000CF911F910F910895E8EDF0E080818F7E36
:101AB0008083E7EDF0E080818160808381E0809326
:101AC000C5020C940C0DE8EDF0E080818C7F8083E2
:101AD0001092E20008951092DA001092E100089549
:101AE0001F920F920FB60F9211240BB60F922F93E5
:101AF0003F934F935F936F937F938F939F93AF9396
:101B0000BF93EF93FF938091E10082FF0BC0809120
:101B1000E20082FF07C08091E1008B7F8093E100AB
:101B20000E946B098091DA0080FF1FC08091D8006D
:101B300080FF1BC08091DA008E7F8093DA00809155
:101B4000D90080FF0DC084E189BD86E189BD09B45B
:101B500000FEFDCF81E08093C6020E94510905C0BE
:101B600019BC1092C6020E9463098091E10080FFB7
:101B700019C08091E20080FF15C08091E2008E7F45
:101B80008093E2008091E20080618093E200809186
:101B9000D80080628093D80019BC85E08093C6028B
:101BA0000E94860A8091E10084FF30C08091E200AB
:101BB00084FF2CC084E189BD86E189BD09B400FEA3
:101BC000FDCF8091D8008F7D8093D8008091E10077
:101BD0008F7E8093E1008091E2008F7E8093E2000F
:101BE0008091E20081608093E2008091C2028823AC
:101BF00011F084E007C08091E30087FD02C081E01E
:101C000001C083E08093C6020E94F10A8091E10046
:101C100083FF29C08091E20083FF25C08091E1000D
:101C2000877F8093E10082E08093C6021092C20217
:101C30008091E1008E7F8093E1008091E2008E7FB1
:101C40008093E2008091E20080618093E20042E0B4
:101C500060E080E00E946C0C8091F00088608093CE
:101C6000F0000E946A09FF91EF91BF91AF919F919F
:101C70008F917F916F915F914F913F912F910F9035
:101C80000BBE0F900FBE0F901F9018951F920F92D2
:101C90000FB60F9211240BB60F922F933F934F93D1
:101CA0005F936F937F938F939F93AF93BF93CF93E4
:101CB000DF93EF93FF93C091E900CF708091EC0028
:101CC000D82FD17080FDD0E81092E9008091F0000B
:101CD000877F8093F00078940E948E0E1092E90026
:101CE0008091F00088608093F000CD2BCF70C0937E
:101CF000E900FF91EF91DF91CF91BF91AF919F915B
:101D00008F917F916F915F914F913F912F910F90A4
:101D10000BBE0F900FBE0F901F9018951F93CF937F
:101D2000DF93CDB7DEB7AA970FB6F894DEBF0FBE2C
:101D3000CDBFE7ECF2E088E08E0F9091F100919337
:101D40008E13FBCF0E94C5098091E80083FF1FC15D
:101D50008091C7029091C802492F50E04A30510546
:101D600008F015C1FA01E95AFF4F0C94B2268038E9
:101D700081F0823809F00BC18091CB028F70809383
:101D8000E9008091EB0085FB882780F91092E9003B
:101D900006C08091C3029091C4029111826090911B
:101DA000E800977F9093E8008093F1001092F10093
:101DB000C8C0282F2D7F09F0EAC0882319F082308F
:101DC00061F0E5C08091C902813009F0E0C0933034
:101DD00009F080E08093C4022BC08091C902811178
:101DE00027C08091CB028F7009F4D1C08093E900A5
:101DF0002091EB0020FF1CC0933021F48091EB0078
:101E0000806214C09091EB0090619093EB0021E010
:101E100030E0A90102C0440F551F8A95E2F74093B4
:101E2000EA001092EA008091EB0088608093EB005A
:101E30001092E9008091E800877F86C08111A7C0D9
:101E40001091C9021F778091E3008078812B8093E5
:101E5000E3008091E800877F8093E8000E94A10C56
:101E60008091E80080FFFCCF8091E3008068809340
:101E7000E300111102C082E001C083E08093C6023A
:101E800086C08058823008F082C08091C90290914B
:101E9000CA028C3D53E0950779F583E08A838AE294
:101EA00089834FB7F894DE01139620E03EE051E2BB
:101EB000E32FF0E050935700E49120FF03C0E29538
:101EC000EF703F5FEF708E2F90E0EA3010F0C79612
:101ED00001C0C0968D939D932F5F243149F74FBF6A
:101EE0008091E800877F8093E8006AE270E0CE018D
:101EF00001960E94AC0B14C0AE014F5F5F4F609122
:101F0000CB020E94F30ABC01892B09F440C09091D6
:101F1000E800977F9093E80089819A810E940D0CD8
:101F20008091E8008B778093E80031C0803879F5A4
:101F30008091E800877F8093E8008091C2028093BF
:101F4000F1008091E8008E778093E8000E94A10C58
:101F50001EC081111CC09091C9029230C0F48091C2
:101F6000E800877F8093E8009093C2020E94A10C52
:101F70008091C202811106C08091E30087FD02C0FA
:101F800081E001C084E08093C6020E94AC09809188
:101F9000E80083FF0AC08091E800877F8093E80013
:101FA0008091EB0080628093EB00AA960FB6F894C4
:101FB000DEBF0FBECDBFDF91CF911F9108959093EB
:101FC000BC018093BB010895E091BB01F091BC017D
:101FD000309721F00190F081E02D099480E0089580
:101FE000EF92FF920F931F93CF93DF93E091BB018A
:101FF000F091BC013097B1F18C010280F381E02DAA
:1020000009958091B10282FF2DC080FF04C08BEC46
:1020100093E00E948F05E80110E285ECE82E83E052
:10202000F82E8091B10280FF0BC088811F928F93A0
:10203000FF92EF920E9428060F900F900F900F9042
:10204000115021961111EDCF8091B10280FF0AC08D
:1020500083EC93E0DF91CF911F910F91FF90EF9070
:102060000C948F05DF91CF911F910F91FF90EF900E
:102070000895E091BB01F091BC01309721F00480FC
:10208000F581E02D09940895CF93DF93EC018091C1
:10209000B9019091BA01C817D90709F1D093BA01D3
:1020A000C093B901E091BB01F091BC013097B9F048
:1020B0000680F781E02DCE0109958091B10282FF63
:1020C0000EC080FF0CC0DF93CF9385EB93E09F930E
:1020D0008F930E9428060F900F900F900F90DF9122
:1020E000CF910895CF93DF93EC018091B701909148
:1020F000B801C817D90709F1D093B801C093B70147
:10210000E091BB01F091BC013097B9F00084F185FA
:10211000E02DCE0109958091B10282FF0EC080FFB3
:102120000CC0DF93CF9385EA93E09F938F930E9437
:1021300028060F900F900F900F90DF91CF91089588
:102140000C944B110E945E1D0C946907BF92CF92B4
:10215000DF92EF92FF920F931F93CF93DF9300D004
:1021600000D01F92CDB7DEB70E9478070EEB11E0CA
:10217000F12C8F2D0E94FF07B82EF801C080C826D1
:1021800039F4F3940F5F1F4FF0E1FF12F2CF30C02C
:102190008091B10281FD0E946711D12CEE24E3945D
:1021A0008E2D8C21F9F0D982FA8281E09E2D9B211F
:1021B00009F480E08B830E94671D8160782F9D83E6
:1021C0008C8349815A816B818D810E949D11498147
:1021D0005A816B817C818D810E94E11CF801908184
:1021E0009E259083D394EE0CF8E0DF12D9CFC9CFAF
:1021F0008FEF89838A831B820E94671D8160782FFD
:102200009D838C8349815A816B818D810E949D11B0
:102210000E94E01C0E94C0201091BD010E94E40FAA
:10222000181741F10E94E40F8093BD019091B10213
:1022300092FF0EC090FF0CC01F928F9386ED93E02B
:102240009F938F930E9428060F900F900F900F90EE
:102250008091BD010F900F900F900F900F90DF9124
:10226000CF911F910F91FF90EF90DF90CF90BF9093
:102270000C94F21C0F900F900F900F900F90DF9125
:10228000CF911F910F91FF90EF90DF90CF90BF9073
:1022900008950C940D080895CF93DF931F92CDB746
:1022A000DEB769830E94FF0790E021E030E069819A
:1022B00002C0220F331F6A95E2F72823392381E0F9
:1022C000232B09F480E00F90DF91CF910895EF92D6
:1022D000FF920F931F93CF93DF938FEE93E00E94B3
:1022E0008F05C0E0D0E08DE2E82E81E0F82E01EE0F
:1022F00013E08C2F0E94FF070E94CA1CFF92EF92EE
:102300001F928F93DF93CF931F930F930E94280602
:1023100021968DB79EB708960FB6F8949EBF0FBE54
:102320008DBFC031D10529F7DF91CF911F910F915A
:10233000FF90EF90089508950895CF93DF93CDB760
:10234000DEB72B970FB6F894DEBF0FBECDBF942F2C
:102350004F83252F588769877A878B874A855B85C6
:10236000452B21F02F3F09F59F3FF9F4DE0111962F
:1023700086E0FD0111928A95E9F785E0FE01379626
:1023800001900D928A95E1F749815A816B817C8198
:102390008D819E810E94E2182B960FB6F894DEBFC5
:1023A0000FBECDBFDF91CF9108954F8158856985CC
:1023B0007A858B850E94E11CD9CFCF93882309F4BD
:1023C000A4C0C82F8CEF8C0F813A48F48C2F0E9448
:1023D0000A2481119AC08C2F0E94BA1B0CC080E283
:1023E0008C0F883058F4C77081E001C0880FCA95FF
:1023F000EAF70E94651CCF910C949F1C8BE58C0F13
:10240000833078F4C53A29F0C63A31F083E890E099
:1024100005C081E890E002C082E890E0CF910C9482
:10242000441088E58C0F853108F06FC0C83A61F11F
:10243000C93A69F1CA3A71F1CB3A79F1CC3A81F1F2
:10244000CD3A89F1CE3A91F1CF3A99F1C13BA1F160
:10245000C03BA9F1C23BB1F1C33BB9F1C43BC1F1EF
:10246000C53BC9F1C63BD1F1C73BD9F1C83BE1F14E
:10247000C93BE9F1CA3BF1F1CB3BF9F1CC3B09F4A3
:102480003FC080E090E03EC082EE90E03BC089EE2D
:1024900090E038C08AEE90E035C085EB90E032C025
:1024A00086EB90E02FC083EB90E02CC084EB90E0B3
:1024B00029C087EB90E026C08CEC90E023C08DEC27
:1024C00090E020C083E891E01DC08AE891E01AC046
:1024D00082E991E017C084E991E014C081E292E0C2
:1024E00011C083E292E00EC084E292E00BC085E26C
:1024F00092E008C086E292E005C087E292E002C066
:102500008AE292E0CF910C947210CF9108958823C3
:1025100029F19CEF980F913A18F40E940D1C0DC000
:1025200090E2980F983058F4877091E001C0990FAD
:102530008A95EAF7892F0E946B1C0C949F1C9BE5DF
:10254000980F933020F480E090E00C944410885A67
:10255000853120F480E090E00C9472100895882377
:1025600021F00E94651C0C949F1C0895882321F083
:102570000E946B1C0C949F1C0895BF92CF92DF9217
:10258000EF92FF920F931F93CF93DF9300D000D071
:1025900000D0CDB7DEB725E0FC01DE011196019039
:1025A0000D922A95E1F7FC014081518102816381FE
:1025B0007481258122952F706115710509F403C37B
:1025C0005F3F19F44F3F09F4FEC26C01862F7D83F3
:1025D0006C83602F782F8D812E830E943E1B182FD5
:1025E000B92E0E943D1B0E942D1AEB2DE295EF7033
:1025F000F0E0EF59FF4F2E810C94B2268B2D807F97
:102600009B2D9F70F92E882319F0F29490EFF922F8
:10261000002349F0FF2009F483C28F2D0E94781C0B
:102620000E949F1C7DC2812F0E948712FF2009F407
:10263000CAC28F2D0E947E1C26960FB6F894DEBF6C
:102640000FBECDBFDF91CF911F910F91FF90EF9003
:10265000DF90CF90BF900C949F1C8B2D807F9B2D83
:102660009F70F92E803219F0F29480EFF822112336
:1026700019F0113009F12AC00023B1F08F2D222367
:1026800051F1213041F526960FB6F894DEBF0FBE0A
:10269000CDBFDF91CF911F910F91FF90EF90DF9011
:1026A000CF90BF900C94881C222319F0213009F49C
:1026B0008AC20E948B1C2DC00023F1F0263008F046
:1026C00082C20E94621C8F2129F023C00023F9F0EE
:1026D000211116C08F2D26960FB6F894DEBF0FBEBF
:1026E000CDBFDF91CF911F910F91FF90EF90DF90C1
:1026F000CF90BF900C94AF12253008F064C209C08F
:10270000F601858180FF0CC28F708583E3CF211194
:102710001CC28F2D83C12B2D26952695237030E06A
:102720002115310521F021303105D1F04CC20023B3
:1027300021F0812F9B2D937002C080E090E02696BF
:102740000FB6F894DEBF0FBECDBFDF91CF911F91C2
:102750000F91FF90EF90DF90CF90BF900C944410BA
:10276000002321F0812F9B2D937002C080E090E028
:1027700026960FB6F894DEBF0FBECDBFDF91CF9186
:102780001F910F91FF90EF90DF90CF90BF900C942E
:102790007210812F002319F00E94461F02C00E9470
:1027A000AE1F26960FB6F894DEBF0FBECDBFDF91E9
:1027B000CF911F910F91FF90EF90DF90CF90BF903E
:1027C0000C9433208B2D837009F07BC00111FBC169
:1027D000812F829586958770880F880F912F9F7023
:1027E000C92ED12CE12CF12C082E04C0CC0CDD1C00
:1027F000EE1CFF1C0A94D2F714FF12C04FE050E009
:1028000060E070E004C0440F551F661F771F8A9573
:10281000D2F7CB01BA01609570958095909503C071
:1028200060E070E0CB012B2D269526952370422F7A
:1028300050E042305105D9F04330510569F16C291F
:102840007D298E299F294130510551F126960FB6D9
:10285000F894DEBF0FBECDBFDF91CF911F910F91D6
:10286000FF90EF90DF90CF90BF900C94521A6C299C
:102870007D298E299F2926960FB6F894DEBF0FBEBC
:10288000CDBFDF91CF911F910F91FF90EF90DF901F
:10289000CF90BF900C946C1A0E94521AC701B601D7
:1028A00026960FB6F894DEBF0FBECDBFDF91CF9155
:1028B0001F910F91FF90EF90DF90CF90BF900C94FD
:1028C000381A002319F08B2D817001C0869588235A
:1028D00009F479C1812F829586958770880F880FBA
:1028E000912F9F70C92ED12CE12CF12C082E04C001
:1028F000CC0CDD1CEE1CFF1C0A94D2F714FF12C096
:102900004FE050E060E070E004C0440F551F661FC8
:10291000771F8A95D2F7CB01BA01609570958095A3
:10292000909503C060E070E0CB012B2D2695269595
:102930002370422F50E042305105D9F04330510509
:1029400069F16C297D298E299F294130510551F16A
:1029500026960FB6F894DEBF0FBECDBFDF91CF91A4
:102960001F910F91FF90EF90DF90CF90BF900C944C
:10297000191B6C297D298E299F2926960FB6F8945C
:10298000DEBF0FBECDBFDF91CF911F910F91FF90A2
:10299000EF90DF90CF90BF900C942B1B0E94191BDF
:1029A000C701B60126960FB6F894DEBF0FBECDBFA5
:1029B000DF91CF911F910F91FF90EF90DF90CF901B
:1029C000BF900C94071B103FD1F128F480E4810FD5
:1029D000803250F0A0C0123F09F462C008F44BC02E
:1029E000133F09F472C097C0F12FF071FF2E8B2DA9
:1029F0008F71002351F00E94A01A812FFF2019F03F
:102A00008295807F68CE8F7066CE0E94C11A812F1A
:102A1000FF2019F08295807F01C08F7026960FB637
:102A2000F894DEBF0FBECDBFDF91CF911F910F9104
:102A3000FF90EF90DF90CF90BF900C94B6120023E0
:102A4000B1F0253008F0BFC08B2D8F7126960FB6E0
:102A5000F894DEBF0FBECDBFDF91CF911F910F91D4
:102A6000FF90EF90DF90CF90BF900C94E61A263045
:102A700008F0A9C0E9CF0023A9F08B2D8F7126960D
:102A80000FB6F894DEBF0FBECDBFDF91CF911F917F
:102A90000F91FF90EF90DF90CF90BF900C94A01A11
:102AA000002359F38B2D8F7126960FB6F894DEBF55
:102AB0000FBECDBFDF91CF911F910F91FF90EF908F
:102AC000DF90CF90BF900C94C11A002399F08B2D0A
:102AD0008F7126960FB6F894DEBF0FBECDBFDF9183
:102AE000CF911F910F91FF90EF90DF90CF90BF900B
:102AF0000C948B1A26960FB6F894DEBF0FBECDBF8E
:102B0000DF91CF911F910F91FF90EF90DF90CF90C9
:102B1000BF900C94861A0023A9F0222309F4ADCFAC
:102B2000812F26960FB6F894DEBF0FBECDBFDF9182
:102B3000CF911F910F91FF90EF90DF90CF90BF90BA
:102B40000C94DD11222309F4ADCF812F26960FB608
:102B5000F894DEBF0FBECDBFDF91CF911F910F91D3
:102B6000FF90EF90DF90CF90BF900C9487124B2D89
:102B70004F70612FC6010E94F01D26960FB6F89483
:102B8000DEBF0FBECDBFDF91CF911F910F91FF90A0
:102B9000EF90DF90CF90BF900C9486194B2D4F7023
:102BA000612FC60126960FB6F894DEBF0FBECDBFCB
:102BB000DF91CF911F910F91FF90EF90DF90CF9019
:102BC000BF900C94F31D26960FB6F894DEBF0FBE8F
:102BD000CDBFDF91CF911F910F91FF90EF90DF90CC
:102BE000CF90BF9008950E94851C0E94541C0E94A3
:102BF0009F1C0E9465210E94332080E090E00E948B
:102C0000441080E090E00C9472100E94751C0C94AB
:102C1000F315CF93DF9300D000D01F92CDB7DEB76E
:102C2000942F4983252F5A836B837C838D834C811A
:102C30005D81452B39F12F3F11F49F3F19F14981F7
:102C40005A816B817C818D810E943E1B292F2295A8
:102C50002F7030E02C30310504F52A3031055CF45A
:102C6000225031092230310568F4853A80F48430ED
:102C700090F4823080F0883E38F4803E60F48450D6
:102C8000813A48F080E014C0803FE1F704C090E250
:102C9000980F983080F781E00BC02C30310521F47B
:102CA00093FB882780F904C02F303105C9F3EACFA0
:102CB0000F900F900F900F900F90DF91CF9108958C
:102CC000CF93DF9300D000D01F92CDB7DEB70F9027
:102CD0000F900F900F900F90DF91CF910895CF93A9
:102CE000DF9300D000D000D0CDB7DEB726960FB668
:102CF000F894DEBF0FBECDBFDF91CF9108951F9333
:102D0000CF93DF93C091CE0116E08091CF01C81719
:102D100099F0D0E01C9FF0011D9FF00D1124E053AD
:102D2000FE4F4081518162817381848195810E942F
:102D30006F162196C770E9CFDF91CF911F9108954B
:102D400040910002509101026091020270910302D1
:102D500080910402909105020C946F1680910502F7
:102D600082958F7009F054C080910202882309F483
:102D70004FC08091CE01A091CF016091000270916F
:102D800001024091030250910402B6E08A1709F44F
:102D90003FC090E041155105C1F17F3F11F46F3FF5
:102DA000A1F1B89FF001B99FF00D1124E053FE4F3F
:102DB000218172132AC02081621327C02281211130
:102DC00024C0238134812417350710F421503109A0
:102DD000241B350B283C3105C0F4209105022F70CF
:102DE00020612093050226E0289FF001299FF00D25
:102DF0001124EB52FE4F80818F708061808380E0D0
:102E000092E00E94BD120C947F1601968770BECF8F
:102E10000895BF92CF92DF92EF92FF920F931F938C
:102E2000CF93DF93CDB7DEB761970FB6F894DEBFCF
:102E30000FBECDBF7C0185E0F701DE011D9601903C
:102E40000D928A95E1F7D7014C9111965C911197FB
:102E50001296DC90129713960D911C911497309155
:102E60000002609101028091030290910402009798
:102E700009F477C16F3F19F43F3F09F472C1B09074
:102E80000202BB2009F4C5C02091050208171907EA
:102E900028F0F801E81BF90BCF0104C0809590954C
:102EA000800F911FCC24C394883C910580F0C12CE5
:102EB000207F09F0CCC0702F198B088B6D2D89896C
:102EC0000E94601680E092E00E94BD12B6C0822F80
:102ED000807F09F047C0651314C0341312C0D110AD
:102EE00010C02F702061209305020E94A01680E080
:102EF00092E00E94BD1280910502D70115968C9335
:102F00002FC00115110519F15F3F11F44F3FF9F082
:102F1000CD2CD1101CC08091CE012091CF0136E084
:102F2000821709F45CC090E0389FF001399FF00DE2
:102F30001124E053FE4F6181561306C06081461391
:102F400003C06281611103C001968770E9CFCD2C67
:102F5000DD2009F426C1809105028160809305027D
:102F6000C12C1FC1651308C0341306C0D11004C0A2
:102F700080910502D701C9C04D875E87DF86702F1B
:102F8000198B088B6D2D89890E9409168823E9F118
:102F9000DD20D9F120910502822F82958F7090E07B
:102FA000029774F0809100029091010298878F83BC
:102FB00019861B870A872C87CE0107960E94BD12AF
:102FC00086E0F701A0E0B2E001900D928A95E1F76A
:102FD0000E94AE160E94A016CC24C394E2C0702FAB
:102FE000198B088B60E089890E943E1B292F22954E
:102FF0002F7030E0223031050CF0C7C09F7009F00F
:10300000C1C0805E883008F4CCC0C7010E94BD12E8
:10301000E3CF0817190708F456C0F801E81BF90BAD
:10302000CF01883C910508F453C0C12C702F198B37
:10303000088B6D2D89890E946016E0E0F2E086E041
:10304000DF011D928A95E9F70E94A016AAC06513B8
:1030500014C0341312C0D11010C080910502F701C2
:103060008583C7010E94BD1286E0E0E0F2E0DF0147
:103070001D928A95E9F7CB2C94C04D875E87DF8639
:10308000702F198B088B6D2D89890E940916882352
:1030900009F4BBCFDD2009F4B8CF20910502822FBF
:1030A00082958F7090E002970CF48ACF8091000295
:1030B000909101029A8389831B821D830C832E8346
:1030C000CE0101967BCF80959095800F911FA9CF5F
:1030D000CD2CDD2009F499CF65132EC034132CC0FC
:1030E0002091050220FD1FC0822F82958F70D9F09C
:1030F000D70115962C9315978F3049F08F5F982F35
:103100009295907F822F8F70892B15968C93C70193
:103110000E94BD1286E0F701A0E0B2E001900D929E
:103120008A95E1F791CF86E0F701A0E0B2E0019047
:103130000D928A95E1F735C04D875E87DF86702F47
:10314000198B088B6D2D89890E940916811138CF42
:1031500080910502816080930502C7010E94BD1223
:1031600020C0DD2009F451CF4D875E87DF86702FA8
:10317000198B088B6D2D89890E940916882309F403
:1031800044CF1ECF81113DCF0CC0243031050CF04F
:103190003CCF9F7009F435CFF7019581907F09F0FE
:1031A00030CF8C2D61960FB6F894DEBF0FBECDBF29
:1031B000DF91CF911F910F91FF90EF90DF90CF9013
:1031C000BF9008951F93CF93DF93CDB7DEB72C97B1
:1031D0000FB6F894DEBF0FBECDBF4F835887698707
:1031E0007A878B879C87CE0107960E9409178823D0
:1031F00069F08F8198852A853B85232BF1F19F3FCC
:1032000009F063C08F3F09F060C037C086E0FE015F
:103210003796DE01119601900D928A95E1F76F8144
:103220007885EA85FB85309741F17F3F11F46F3F48
:1032300021F12091CF0130E0C901019687709927D3
:103240004091CE0150E08417950709F447C0698387
:103250007A83FD83EC8396E0929FD001939FB00D1B
:103260001124A053BE4FFE01319601900D929A9504
:10327000E1F78093CF010E947F1616E08091CE0186
:103280009091CF018917C1F1189FC001112480537B
:103290009E4F0E940917882379F1E091CE011E9F6D
:1032A000F0011124E053FE4F40815181628173810E
:1032B000848195810E946F168091CE0190E00196E5
:1032C000877099278093CE01D9CF4F815885698522
:1032D0007A858B859C850E946F16CFCF0E9405163C
:1032E0001092CF011092CE01E0E0F2E086E0DF0123
:1032F0001D928A95E9F7C1CF2C960FB6F894DEBFE0
:103300000FBECDBFDF91CF911F910895DF92EF9255
:10331000FF920F931F93CF93DF93FC01892B09F446
:103320008AC0E12CF12CDD24D394EF012196849105
:10333000853709F461C058F4843708F04EC08430F2
:1033400008F06AC08130D1F0823071F174C08837E2
:1033500009F45DC050F4863709F455C0873709F089
:103360006AC08E2D0E94721C54C09CE7980F903743
:1033700008F061C08F770E94871250C08F010E5FE6
:103380001F4FFE01849190E2980F983050F487709F
:10339000FD2D01C0FF0F8A95EAF78F2F0E94781C40
:1033A00014C00E94DD1113C08F010E5F1F4FFE017C
:1033B000C49180E28C0F883060F4C7708D2D01C0FD
:1033C000880FCA95EAF70E947E1C0E949F1CE801A4
:1033D00025C08C2F0E948712FACF9F012E5F3F4F8E
:1033E000FE01C491CC2369F08FE99FE00197F1F7CA
:1033F00000C00000C150F6CF9F012E5F3F4FFE017D
:10340000F490E9010BC00E94621CE82E07C00E94E4
:10341000751C0E949F1C02C00E94DD118F2D882305
:1034200041F0EFE9FFE03197F1F700C00000815073
:10343000F6CFFE017ACFDF91CF911F910F91FF90D0
:10344000EF90DF90089560938602709387028093D7
:103450008802909389020C94F11C089560938A026B
:1034600070938B0280938C0290938D020C94F01CCD
:103470000F931F9300918A0210918B0220918C026E
:1034800030918D02602B712B822B932B60938A02DB
:1034900070938B0280938C0290938D021F910F91F9
:1034A0000C94F01C0F931F9300918A0210918B02D1
:1034B00020918C0230918D0260237123822393230B
:1034C00060938A0270938B0280938C0290938D029A
:1034D0001F910F910C94F01C0F931F9300918A027F
:1034E00010918B0220918C0230918D026027712700
:1034F0008227932760938A0270938B0280938C02B9
:1035000090938D021F910F910C94F01C60E070E07D
:10351000CB010C94231A0F931F9341E050E060E01D
:1035200070E08A019B0104C0000F111F221F331F8E
:103530008A95D2F7C901B8011F910F910C94231AF3
:103540000F931F9341E050E060E070E004C0440F2F
:10355000551F661F771F8A95D2F78091860290913A
:103560008702A0918802B09189028A019B01082BF1
:10357000192B2A2B3B2BC901B8011F910F910C94D9
:10358000231A0F931F9341E050E060E070E004C005
:10359000440F551F661F771F8A95D2F740955095A7
:1035A000609570958091860290918702A091880223
:1035B000B09189028A019B01082319232A233B2306
:1035C000C901B8011F910F910C94231A0F931F93F7
:1035D00041E050E060E070E004C0440F551F661FFA
:1035E000771F8A95D2F78091860290918702A091E9
:1035F0008802B09189028A019B01082719272A278E
:103600003B27C901B8011F910F910C94231A0F9306
:103610001F930091860210918702209188023091B9
:103620008902602B712B822B932B1F910F910C948D
:10363000231A0F931F930091860210918702209105
:1036400088023091890260237123822393231F9182
:103650000F910C94231A0F931F93009186021091DF
:103660008702209188023091890260277127822782
:1036700093271F910F910C94231A08958F929F9274
:10368000AF92BF92DF92EF92FF920F931F93CF936F
:10369000DF9300D000D01F92CDB7DEB76B837C8361
:1036A0008D838A018C819D81892B21F01F3F29F414
:1036B0004F3F19F480E090E04CC08B818823C9F122
:1036C00080908A0290908B02A0908C02B0908D0224
:1036D0008091860290918702A0918802B091890220
:1036E000882A992AAA2ABB2A8FE1E82EF12CD50133
:1036F000C4010E2C04C0B695A795979587950A949A
:10370000D2F780FF07C0DE2CB8018E2D0E940F1E5D
:10371000019729F481E0E81AF10848F7D12C88E0F4
:10372000189FF0011124E00FF11DEA5FFD4FD082D8
:1037300009C088E0189FF0011124E00FF11DEA5F35
:10374000FD4FD08009831A8369817A818D2D0E9473
:103750000F1E0F900F900F900F900F90DF91CF9151
:103760001F910F91FF90EF90DF90BF90AF909F90CF
:103770008F90089590910A01992321F090910B0167
:10378000911109C020910C0130910D01F90132967F
:103790009FEF40E030C0982F9695969596959F3173
:1037A000A0F4E0910C01F0910D01E90FF11D87707B
:1037B00021E030E0A90102C0440F551F8A95E2F7CD
:1037C000CA019181892B818308959091B10290FF64
:1037D00023C01F928F938BE194E09F938F930E945D
:1037E00028060F900F900F900F9008959F3F39F08B
:1037F0004F5F4E3141F051915813F8CF0DC0511128
:10380000F7CF942FF5CF9F3F39F0F901E90FF11D64
:1038100097FDFA9582830895089590910A0199235E
:1038200021F090910B01911109C020910C01309170
:103830000D01F9013296205E3F4F30C0982F9695CA
:10384000969596959F31A8F4E0910C01F0910D01A9
:10385000E90FF11D877021E030E0A90102C0440F9B
:10386000551F8A95E2F7CA0180959181892381834A
:1038700008959091B10290FF16C01F928F938DEF23
:1038800093E09F938F930E9428060F900F900F90C4
:103890000F9008953196E217F30729F0908198135D
:1038A000F9CF1082F7CF089581E090E0E0910C010C
:1038B000F0910D01E80FF91F1082019680329105F9
:1038C000A9F708958091B00208959091B002892BD4
:1038D0008093B002089580959091B00289238093DF
:1038E000B00208958093B00208951092B002089536
:1038F0009091AF02892B8093AF02089580959091AB
:10390000AF0289238093AF0208951092AF02089509
:1039100080938E02089510928E02089580910C017A
:1039200090910D01FC0131969C01205E3F4F80E09B
:10393000919191118F5FE217F307D1F70895E0910C
:103940000C01F0910D018091B0028083E0910C0197
:10395000F0910D0190818091AF02892B808380913D
:103960008E02882361F0E0910C01F0910D019081AD
:10397000892B80830E948E1C811110928E0280916F
:103980000C0190910D010C94F00F909339018093EC
:10399000380108958295982F9C7C392F369536955D
:1039A000282F237344E0249FC0011124932F982BC8
:1039B000292F2A7A2695892F8575880F822B0895BD
:1039C0000895CF93DF9300D000D01F92CDB7DEB71C
:1039D0000F900F900F900F900F90DF91CF9108955F
:1039E000089508950C9449118091C602843021F104
:1039F0001092B20220E488E190E00FB6F894A89506
:103A0000809360000FBE2093600083B7817F846045
:103A100083BF83B7816083BF7894889583B78E7F97
:103A200083BF0FB6F894A895809160008861809359
:103A30006000109260000FBE0895CF930E949B110A
:103A40000E9478070E949C11C0E08C2F0E94FF0703
:103A5000811104C0CF5FC031C1F701C081E0CF91B7
:103A600008950E9405080C9405161F920F920FB638
:103A70000F9211248F939F93AF93BF938091B202C3
:103A8000811113C08091B3029091B402A091B5024C
:103A9000B091B6024196A11DB11D8093B3029093DF
:103AA000B402A093B502B093B602BF91AF919F91BB
:103AB0008F910F900FBE0F901F90189582E084BDDC
:103AC00093E095BD9AEF97BD80936E0008952FB750
:103AD000F8948091B3029091B402A091B502B09194
:103AE000B6022FBF08952FB7F8946091B30270917A
:103AF000B4028091B5029091B6022FBF0895CF9283
:103B0000DF92EF92FF920F931F932FB7F89440919B
:103B1000B3025091B4026091B5027091B6022FBF0A
:103B20006A017B01EE24FF248C0120E030E0C01606
:103B3000D106E206F30610F4415051099A01281B00
:103B4000390BC9011F910F91FF90EF90DF90CF903B
:103B500008951F920F920FB60F9211248F939F9387
:103B6000AF93BF938091B3029091B402A091B5023C
:103B7000B091B6020196A11DB11D8093B30290933E
:103B8000B402A093B502B093B602BF91AF919F91DA
:103B90008F910F900FBE0F901F9018950E94F20CFE
:103BA000F8942FEF87EA91E6215080409040E1F7AA
:103BB00000C0000087E090EBDC018093CF0290937F
:103BC000D002A093D102B093D2029CE088E10FB65C
:103BD000F894A895809360000FBE90936000FFCF8B
:103BE00080E090E008950895E72FF0E090E1899F4C
:103BF000E00DF11D112483E0EE0FFF1F8A95E1F720
:103C0000E60FF11DEE51FF4F84910895E82FF0E08B
:103C1000EE0FFF1FEE59F0408591949108950E9498
:103C2000F41D90E4980F903218F40E94061E089537
:103C30008D3B50F4883AA0F5853A28F5843000F59C
:103C4000813009F49DC099C0883E98F4803EC0F44C
:103C50008F3B09F092C00E9405162FEF80E792E09B
:103C6000215080409040E1F700C000000E94CE1D2E
:103C700084C0803F08F481C0282F30E0306582C0C6
:103C8000282F30E07FC0853A29F0863A31F023E8CA
:103C900030E478C021E830E475C022E830E472C036
:103CA000883A61F1893A69F18A3A71F18B3A79F18E
:103CB0008C3A81F18D3A89F18E3A91F18F3A99F1EE
:103CC000813BA1F1803BA9F1823BB1F1833BB9F18A
:103CD000843BC1F1853BC9F1863BD1F1873BD9F1EA
:103CE000883BE1F1893BE9F18A3BF1F18B3BF9F14A
:103CF0008C3B09F43FC020E034E444C022EE34E4BD
:103D000041C029EE34E43EC02AEE34E43BC025EB4A
:103D100034E438C026EB34E435C023EB34E432C05D
:103D200024EB34E42FC027EB34E42CC02CEC34E437
:103D300029C02DEC34E426C023E835E423C02AE86A
:103D400035E420C022E935E41DC024E935E41AC079
:103D500021E236E417C023E236E414C024E236E45C
:103D600011C025E236E40EC026E236E40BC027E29D
:103D700036E408C02AE236E405C020E030E002C0A4
:103D800021E030E0C90108958091B90280FF0BC0A5
:103D90006091110185E0689FB001112475956795C8
:103DA000759567952BC081FF09C06091110185E071
:103DB000689FB00111247595679520C082FF07C0E8
:103DC0006091110185E0689FB001112417C09091A6
:103DD000BA029923D1F060911001961788F72091CB
:103DE000110185E0289F90011124929FA001939FCB
:103DF000500D112470E0CA010E949E2660387105A2
:103E000040F46115710539F002C065E070E0862F5D
:103E100008958FE7089581E008958091B90280FFA9
:103E200008C060910F0170E075956795759567956D
:103E300021C081FF06C060910F0170E07595679504
:103E400019C082FF04C060910F0170E010C0909112
:103E5000BA029923C1F060910E019617A0F78091E4
:103E60000F01899FC001112470E00E949E266038D6
:103E7000710528F46115710521F0862F08958FE7EB
:103E8000089581E0089561E070E0F4CF803F21F46F
:103E90000E94C41E819504C0813F29F40E94C41E63
:103EA0008093BD020895823F21F40E94C41E819533
:103EB00004C0833F29F40E94C41E8093BC0208956D
:103EC000893F19F40E940D1F05C08A3F31F40E94FA
:103ED0000D1F81958093BE0208958B3F21F40E94AF
:103EE0000D1F819504C08C3F29F40E940D1F809303
:103EF000BF020895843F21F48091BB02816017C006
:103F0000853F21F48091BB02826011C0863F21F47D
:103F10008091BB0284600BC0873F21F48091BB027B
:103F2000886005C0883F31F48091BB028061809336
:103F3000BB0208958D3F21F48091B90281600BC0CE
:103F40008E3F21F48091B902826005C08F3F29F431
:103F50008091B90284608093B9020895803F39F45A
:103F60008091BD0287FF6CC01092BD0269C0813F85
:103F700029F48091BD021816BCF362C09091BC0276
:103F8000823F29F497FF5CC01092BC0259C0833F66
:103F900019F41916CCF354C0893F41F48091BE0244
:103FA00018160CF04DC01092BE024AC08A3F29F488
:103FB0008091BE0287FF44C0F6CF8B3F39F48091D9
:103FC000BF0287FF3DC01092BF023AC08C3F29F468
:103FD0008091BF021816BCF333C0843F21F4809156
:103FE000BB028E7F17C0853F21F48091BB028D7F7D
:103FF00011C0863F21F48091BB028B7F0BC0873FAD
:1040000021F48091BB02877F05C0883F31F4809105
:10401000BB028F7E8093BB0213C08D3F21F4809141
:10402000B9028E7F0BC08E3F21F48091B9028D7F43
:1040300005C08F3F29F48091B9028B7F8093B9022C
:104040008091BC0281110EC08091BD0281110AC015
:104050008091BE02811106C08091BF02811102C011
:104060001092BA0208958091B10283FF7EC080E66B
:1040700094E00E948F058091BB021F928F938BE585
:1040800094E09F938F930E94280689E594E00E9414
:104090008F058091BC02282F082E000C330B3F9314
:1040A0008F9386E594E09F938F930E94280684E582
:1040B00094E00E948F058091BD02282F082E000CED
:1040C000330B3F938F9381E594E09F938F930E94EE
:1040D00028068FE494E00E948F058091BE02282F6D
:1040E000082E000C330B3F938F938CE494E09F9346
:1040F0008F930E9428068AE494E00E948F058091A5
:10410000BF02282F082E000C330B3F938F9387E4B8
:1041100094E09F938F930E94280684E494E00E9489
:104120008F058091BA021F928F9381E494E09F9350
:104130008F930E9428068FE394E00E948F05809160
:10414000B9021F928F938CE394E09F938F930E9408
:10415000280689E394E00E948F058DB79EB74C96A0
:104160000FB6F8949EBF0FBE8DBF8BEB92E00E94FE
:1041700039100E94671D9093B8028093B70208958A
:104180001F93CF93DF938091B7029091B8020E9462
:104190007F1DAC019091BA02992321F02091120168
:1041A00030E006C0209113018AE0289F900111247D
:1041B0004217530708F485C08091BC02C091BD022C
:1041C000D091BE021091BF02811107C0C11175C00C
:1041D000D11173C0111171C074C09F3F19F09F5F5E
:1041E0009093BA02181624F40E94C41E8093BC0255
:1041F0008091BC0287FF05C00E94C41E81958093F8
:10420000BC021C1624F40E94C41E8093BD0280913F
:10421000BD0287FF05C00E94C41E81958093BD0228
:104220006091BC02662331F1C091BD02CC2311F133
:10423000062E000C770B880B990B0E94992523E31F
:1042400033E343E35FE30E94FD250E946125609311
:10425000BC026C2FCC0F770B880B990B0E94992511
:1042600023E333E343E35FE30E94FD250E946125DE
:104270006093BD021D1624F40E940D1F8093BE02A0
:104280008091BE0287FF05C00E940D1F819580931B
:10429000BE02111624F40E940D1F8093BF0280916C
:1042A000BF0287FF05C00E940D1F81958093BF024A
:1042B000DF91CF911F910C9433209F3F09F08FCF56
:1042C00097CFDF91CF911F910895EBEBF2E085E05E
:1042D000DF011D928A95E9F71092BA021092B90295
:1042E000089583E896E00E948F051F9281E08F93E6
:1042F0001F9285E08F9385E396E09F938F930E94B2
:1043000028060F900F900F900F900F900F90089528
:104310008330E9F128F4813061F0823009F10895A9
:10432000853009F462C008F449C0863009F474C0CD
:10433000089580911301262F30E0280F311D2F3F63
:10434000310524F4680F6093130103C08FEF80934D
:104350001301809113011F928F938EE695E072C036
:1043600080911201262F30E0280F311D2F3F31059B
:1043700024F4680F6093120103C08FEF8093120141
:10438000809112011F928F938CE595E05BC0809124
:104390001101262F30E0280F311D2F3F310524F465
:1043A000680F6093110103C08FEF8093110180911A
:1043B00011011F928F9389E495E044C08091100110
:1043C000262F30E0280F311D2F3F310524F4680FD0
:1043D0006093100103C08FEF809310018091100152
:1043E0001F928F9384E395E02DC080910F01262FBB
:1043F00030E0280F311D2F3F310524F4680F609302
:104400000F0103C08FEF80930F0180910F011F9266
:104410008F938BE195E016C080910E01262F30E03E
:10442000280F311D2F3F310524F4680F60930E01D2
:1044300003C08FEF80930E0180910E011F928F9326
:1044400080E095E09F938F930E9428060F900F9035
:104450000F900F900895833081F128F4813059F046
:104460008230D1F00895853009F449C0B8F1863022
:1044700009F456C0089580911301681720F4861B33
:104480008093130102C010921301809113011F92B7
:104490008F9381EF94E054C080911201681720F44B
:1044A000861B8093120102C01092120180911201AA
:1044B0001F928F938FED94E043C080911101681794
:1044C00020F4861B8093110102C01092110180918B
:1044D00011011F928F938CEC94E032C080911001F7
:1044E000681720F4861B8093100102C010921001FF
:1044F000809110011F928F9387EB94E021C08091EF
:104500000F01681720F4861B80930F0102C01092E0
:104510000F0180910F011F928F938EE994E010C0DC
:1045200080910E01681720F4861B80930E0102C053
:1045300010920E0180910E011F928F9383E894E0F8
:104540009F938F930E9428060F900F900F900F90CB
:104550000895CF93C82F1F928F9388E897E09F9379
:104560008F930E94280681E090E0A0E0B0E0BC01BB
:10457000CD0104C0660F771F881F991FCA95D2F717
:104580000E942E1A0F900F900F900F90CF910C94C5
:104590000516CF938732A8F58E3108F02BC18031F4
:1045A00009F49FC0F8F4873009F464C0A8F4863099
:1045B00009F024C18091B102817F8E7F8093B10286
:1045C0008DE897E00E948F058BE69AE00E948F05A8
:1045D00081E08093C1024CC08B30F1F18E3009F440
:1045E0006CC00CC1863109F4B0C020F4813109F4EB
:1045F000EDC004C1893109F491C08B3109F449C07F
:10460000FDC0883349F150F4893209F4F1C0853393
:1046100009F4EEC0873209F0F1C0EAC0833409F42E
:10462000E7C028F48A3308F4E9C08953E4C0883429
:1046300009F0E4C00E9405168AE59AE00E948F0501
:104640002FEF83ED90E3215080409040E1F700C0D0
:1046500000000E94CE1D0CC084EB97E05CC081E49A
:104660009AE00E948F058091B10281608093B1022F
:10467000C1E0C9C08091B102C82FC17080FFEFCFE7
:104680008DE49AE00E948F058091B102817F8E7F38
:104690003DC09091B10291FBCC27C0F981E0C827C1
:1046A000892FC0FB81F98093B102CC2319F084E3F8
:1046B0009AE027C086E29AE02EC09091B10292FB68
:1046C000CC27C0F981E0C827892FC0FB82F98093ED
:1046D000B102CC2319F087E19AE013C087E09AE099
:1046E0001AC09091B10293FBCC27C0F981E0C82792
:1046F000892FC0FB83F98093B102CC2351F08BEF5B
:1047000099E00E948F058091B10281608093B1028F
:104710007AC08EEE99E00E948F05AACF8FED99E0C6
:104720000E948F058DEB99E00E948F0589E799E043
:104730000E948F058CE499E00E948F0581E199E049
:104740000E948F0582EE98E0E6CF84ED98E00E940B
:104750008F050E94E40F1F928F938AEB98E09F933E
:104760008F930E94280680910A011F928F9383EAFB
:1047700098E09F938F930E9428068091B6011F9224
:104780008F9380E998E09F938F930E9428068091F1
:104790000B011F928F938DE798E09F938F930E9458
:1047A00028060E94731D9F938F937F936F9386E6D5
:1047B00098E09F938F930E9428068DB79EB74696E8
:1047C0000FB6F8949EBF0FBE8DBF52CF0E94051644
:1047D000C0910B0181E0C827C0930B01CC2329F0C5
:1047E0008CE598E00E948F050EC081E598E093CF9C
:1047F00080E001C08D510E94A9223ACF8FE498E059
:104800000E948F05C0E08C2FCF91089580E008951D
:1048100080E00895CF93C82F8091C102813079F054
:1048200020F0823009F44DC044C1E0910C01F091B8
:104830000D0180818152823008F03DC108C0E091B5
:104840000C01F0910D0180818152823060F48C2F37
:104850000E940624811104C08C2F0E94C9222FC0FF
:1048600081E090E02CC08C2F0E940824811126C08A
:10487000C431E1F070F4CB3081F0C031D1F40E944A
:10488000712180E897E00E948F0582E08093C10249
:1048900015C0C93259F0C83361F48DE897E00E9421
:1048A0008F0584E897E00E948F0508C01092C1022E
:1048B00004C18EE797E00E948F05FFC081E0817000
:1048C000FEC0C43228F5CE3108F0C1C0CB30A1F112
:1048D000D0F4C73009F0D3C08EE18093130182E396
:1048E000809312018AE08093110184E1809310018A
:1048F00088E080930F0188E280930E0184E296E0C5
:104900000E948F05BFC0C33149F1C431C1F0B7C0A7
:10491000CB3409F4A9C028F4C93289F0C83361F056
:10492000AEC0C13509F49EC0C23509F499C0CE3479
:1049300009F0A5C06AE09EC00E947121A3C08091C9
:10494000C002882319F01092C0029CC081E396E057
:104950000E948F0581E08093C102B1C08BE096E098
:104960000E948F0589EF95E00E948F0580911301C9
:104970001F928F9386EF95E09F938F930E94280656
:1049800084EF95E00E948F0582EE95E00E948F05EE
:10499000809112011F928F938FED95E09F938F93DB
:1049A0000E9428068DED95E00E948F058EEC95E023
:1049B0000E948F05809111011F928F938BEC95E0DF
:1049C0009F938F930E94280689EC95E00E948F05A3
:1049D00088EB95E00E948F05809110011F928F93C4
:1049E00085EB95E09F938F930E94280683EB95E0DB
:1049F0000E948F058EE995E00E948F0580910F013E
:104A00001F928F938BE995E09F938F930E942806C6
:104A100089E995E00E948F0582E895E00E948F0564
:104A200080910E011F928F938FE795E09F938F9354
:104A30000E9428068DE795E00E948F058DB79EB7EE
:104A400048960FB6F8949EBF0FBE8DBF1BC0CE51C7
:104A5000EC2FF0E0E25DFE4F80818093C00212C037
:104A600061E003C061E006C06AE08091C0020E947C
:104A7000882108C08091C0020E942B2203C082E2DC
:104A800096E013C08091C002882369F01F928F9333
:104A90008CE196E09F938F930E9428060F900F90D1
:104AA0000F900F9004C089E196E00E948F0581E08D
:104AB00006C01092C10280E002C080E000CFCF911A
:104AC00008950E9468256894B1110C94F725089503
:104AD0000E94DC2588F09F5798F0B92F9927B7518D
:104AE000B0F0E1F0660F771F881F991F1AF0BA9592
:104AF000C9F714C0B13091F00E94F625B1E00895D5
:104B00000C94F625672F782F8827B85F39F0B93FC6
:104B1000CCF3869577956795B395D9F73EF4909544
:104B20008095709561957F4F8F4F9F4F0895E894C2
:104B300009C097FB3EF490958095709561957F4FE5
:104B40008F4F9F4F9923A9F0F92F96E9BB27939593
:104B5000F695879577956795B795F111F8CFFAF4A3
:104B6000BB0F11F460FF1BC06F5F7F4F8F4F9F4FD4
:104B700016C0882311F096E911C0772321F09EE832
:104B8000872F762F05C0662371F096E8862F70E098
:104B900060E02AF09A95660F771F881FDAF7880F72
:104BA0009695879597F9089557FD9058440F551F8E
:104BB00059F05F3F71F04795880F97FB991F61F09F
:104BC0009F3F79F087950895121613061406551F16
:104BD000F2CF4695F1DF08C0161617061806991F82
:104BE000F1CF86957105610508940895E894BB2777
:104BF00066277727CB0197F908950E9410260C9419
:104C000081260E94732638F00E947A2620F0952390
:104C100011F00C946A260C94702611240C94F7253C
:104C20000E94D42570F3959FC1F3950F50E0551F56
:104C3000629FF001729FBB27F00DB11D639FAA27F1
:104C4000F00DB11DAA1F649F6627B00DA11D661F40
:104C5000829F2227B00DA11D621F739FB00DA11D61
:104C6000621F839FA00D611D221F749F3327A00D1B
:104C7000611D231F849F600D211D822F762F6A2FB7
:104C800011249F5750409AF0F1F088234AF0EE0F1C
:104C9000FF1FBB1F661F771F881F91505040A9F749
:104CA0009E3F510580F00C946A260C94F7255F3FD7
:104CB000E4F3983ED4F3869577956795B795F79585
:104CC000E7959F5FC1F7FE2B880F911D96958795FD
:104CD00097F9089597F99F6780E870E060E008957C
:104CE0009FEF80EC089500240A9416161706180604
:104CF0000906089500240A941216130614060506E0
:104D00000895092E0394000C11F4882352F0BB0F70
:104D100040F4BF2B11F460FF04C06F5F7F4F8F4FD3
:104D20009F4F0895991B79E004C0991F961708F0CA
:104D3000961B881F7A95C9F78095089597FB072ED3
:104D400016F4009407D077FD09D00E94BB2607FC1B
:104D500005D03EF4909581959F4F0895709561958B
:104D60007F4F0895EE0FFF1F0024001C0BBE07901D
:104D7000F691E02D0994AA1BBB1B51E107C0AA1FA5
:104D8000BB1FA617B70710F0A61BB70B881F991FEC
:104D90005A95A9F780959095BC01CD010895F89496
:024DA000FFCF43
:104DA2000E08FF08DC08A808740801018F02280811
:104DB200140A321E404D36223965031803E202C03E
:104DC200028702FA0113022C024502650200010267
:084DD2000304050607080900AF
:00000001FF
